:1000000000308A00BB2E0000831A0A28A500030EC8
:10001000A6000F288312A500030EA600A614A50EA5
:100020000408A7002008A8002108A9002208AA00A7
:100030002308AB002408AC0083120B1E21288B1868
:1000400008298B1E25280B191A292708840028083F
:10005000A0002908A1002A08A2002B08A3002C0850
:10006000A400260E83008312250EA618831609000D
:100070000A108A100A11820711347B34253429347E
:100080004B348934C1343B3401340B34FF34BF3436
:10009000EF34FD340A108A100A1182076334613488
:1000A0006C3420343D34203400340A108A100A1194
:1000B0008207313439342D344A3455344C342D349C
:1000C0003034353400340A108A100A118207233480
:1000D000203444346F3477346E346C346F3461348C
:1000E000643400340A108A100A1182072334203441
:1000F00044346934733470346C346134793400348A
:100100000A108A100A1182072334203441345034F3
:100110005234533400340A108A100A1182072334EF
:10012000203449346E34763461346C346934643448
:1001300000340A108A100A11820720346D346F349B
:100140006434653400340A108A100A11820764345A
:1001500028346F34293477346E346C346F3461341E
:1001600064342C34203464342834693429347334AE
:1001700070346C346134793400340A108A100A11F6
:1001800082072834613429345034523453340034D3
:100190000A108A100A1182075034493443340D344E
:1001A00000340A108A100A1182073A344B34423460
:1001B0003034543448344E342D34453420343A34B9
:1001C0006A346A344034613470347234733477344E
:1001D0006F3472346C3464342E346E346534743459
:1001E00020345734583420345334743461347234E6
:1001F0007434753470342034283400340A148A106E
:100200000A11820763346D3464343A342034003484
:100210008B12AE0A8B168B108A112528B6010A3074
:100220005E02031C17290A30DE02B60A0F295E0897
:10023000B70000348B12B00B2B290B122F08B00023
:100240002E08B10031083202031828293108B20003
:10025000AE01B5140B16BD0803193029BD033E29A4
:100260008316851700308312851B01300038031D6B
:100270003E29B30A0319B40AFF30BD002D1CB6296C
:10028000B51C8429B510BE08031D4D290B30B600DE
:100290000A30B7000130BE00842901303E02031D40
:1002A0005B293108DE000E213608B8003708B90096
:1002B0000230BE00842902303E02031D66290C3044
:1002C000B6000A30B7000330BE00842903303E0276
:1002D000031D70293208DE000E210430BE0084297F
:1002E00004303E02031D7B290D30B6000A30B700F2
:1002F0000530BE00842905303E02031D84293B08D9
:10030000B7003A08B600BE01003035180130003899
:10031000031D9B2935148316851083128514370815
:10032000DE005E083820A100210886008316051132
:1003300083120511B6293510831605118312051590
:10034000B608031DAB290A30DE005E083820A10084
:1003500021088600B2293608DE005E083820A10098
:100360002108860083168510831285108B160B11C9
:100370008A11252807309F00831605088500033061
:100380008312A000A00BC2291F080C130030F839FB
:10039000031987109D0183169F018312D62E4808EA
:1003A00083169B009C131C141A088312A1000034AE
:1003B00081010430A000A01DE529073081018130B2
:1003C00084000008C0390F38800064008130840048
:1003D0000008C039200480008B160B16C0308B0437
:1003E000E22E0408A1000830A000831685158312B0
:1003F000851DF829C401A0170D2AA0130D2A03108A
:10040000C40C851DC41720170D2A2013A00BFF292B
:10041000210884004408A100222A01308400003011
:10042000A01B5530A100A10B132A840B0F2A0D30FD
:10043000A01B0330A100A10B1B2AA01BFD29201B20
:10044000052AFF2900345630840000080319372A92
:100450000130A100A001A00B2B2AA10B2A2A4A30AF
:10046000A000A00B312A00000000800B282A0034D5
:1004700083160510831205140830A1000000000047
:100480000000A117532AA113D80C03180510031C50
:1004900005142117532A2113A10B442A0000000040
:1004A00000000510532A0130A0008401840B562A55
:1004B000A00B552A0E308400840B5C2AA11B432A12
:1004C000211B4B2A0034430883169B0083124408E7
:1004D00083169A009C131C1583120B138B138B1B12
:1004E0006E2A553083169D00AA309D009C14C030A2
:1004F00083128B040A30D60023220034C208031D65
:10050000972AF1212108C2000A30D600232242088E
:10051000D800382241304202031C952A5B30420247
:100520000318952A42082038962A4208C2000D3046
:10053000D80038220A30D80038226F304202031D1A
:10054000AE2AC30143086320C30AD80038220A3008
:100550004302031DA22A0930AD00E32A693042029A
:10056000031DBF2AC30143087220C30AD8003822E2
:1005700009304302031DB32A0B30AD00E32A61307A
:100580004202031DD02AC30143088020C30AD800B9
:10059000382206304302031DC42A1930AD00E32A75
:1005A000C30143088B20C30AD80038220930430214
:1005B000031DD12A0D30D80038220A30D800382245
:1005C0000130A100FA2AC30143089920C30AD800C8
:1005D000382205304302031DE42A0D30D8003822AA
:1005E0000A30D80038220230C3002D08C40063222C
:1005F0000030A10000340B138B138B1BFC2A00303E
:100600008A0000280034C308031D092BC2080319FF
:10061000152B0430C400FA30D6002322C40B0B2B58
:1006200042080319C303C203032B0034CB01643017
:100630004902031C1F2B6430C902CB0A172BCB08BD
:10064000031D252BCA0803192B2B30304B07CC0078
:100650004C08D8003822CB010A304902031C342B45
:100660000A30C902CB0A2C2BCB08031D3A2BCA082F
:100670000319402B30304B07CC004C08D8003822EF
:1006800030304907CC004C08D8003822003483169B
:10069000051383120513EF30A000A00B4D2B0000B3
:1006A000000083160513831205178316051783129E
:1006B000051B5D2B0030A100752B1630A000A00B90
:1006C0005F2B831605178312051F692B0030A100CD
:1006D000752B9530A000A00B6B2B0000000083163B
:1006E0000513831205170130A1000034D60108302C
:1006F000560203189A2B8316051383120513033031
:10070000A000A00B812B0310D50C0318892B051317
:100710008A2B05178316051310308312A000A00B37
:100720008F2B0000831605138312051700000000AD
:10073000D60A772B0034560858068039DA00D61FBF
:10074000A62BD509D609D50A0319D60AD81FAD2B71
:10075000D709D809D70A0319D80A1030A000A30175
:10076000D901D60CD50C031CBB2B5708A3070318C3
:10077000D90A5808D907D90CA30CA20CA10CA00BBC
:10078000B12BDA1FC82BA109A209A10A0319A20AD9
:100790000000E62C64303102031CD12B3130C20042
:1007A000D32B3030C2002130D80038226B30C50046
:1007B000C6014508C800CF212108C700C708031D8E
:1007C000E22BE72B4708D8003822C50AD92B461C54
:1007D000EF2B0D30D80038220A30D80038220330F1
:1007E000C5003030D8003822C50BF12B2F30D8008F
:1007F00038224208D800382230303807C500450872
:10080000D800382230303907C5004508D8003822D2
:100810000B138B138B1B092C6730D800382232083E
:10082000C9000130CA001623B2017430D800382242
:10083000C0308B04D401D40A0B138B138B1B1D2CDB
:1008400047232108C800CC30D50076234430D5009A
:100850007623C0308B0483160513831205170330EB
:10086000D500FA30D6002322D50B312C0B138B1375
:100870008B1B372C47232108C807CC30D5007623A3
:10088000BE30D5007623D3010930530203187E2CE5
:100890004A305307D500D601083056020318762C8B
:1008A0008316051383120513000000000000831651
:1008B0000513831205170330A000A00B5D2C000068
:1008C000831605178312051B672C0310682C03146D
:1008D000D70C1030A000A00B6B2C00008316051362
:1008E0008312051700000000D60A4C2C5708A100FF
:1008F0005508840021088000D30A442CC0308B04A2
:1009000006305402031C912C0330D5002E30D80041
:100910003822D50B862C0D30BA000D30BB00672D68
:10092000962C023048020319962C1B2C4A30D50015
:100930000930D600D701DB0156085B020318C72C2B
:10094000DC0108305C020318C52C5B0855078400E5
:100950000008A0005C08A1000319B22C0310A00C31
:10096000A10BAE2C20080139D80057080139D90055
:10097000580859060139DA000310D70CDA080319B0
:10098000C32C8C30D706DC0AA12CDB0A9C2C570820
:10099000A100A1080319CD2C1B2CC6014A08C500D3
:1009A000CB1CDC2CC6174617C6164616C6154615B0
:1009B000C61446144714DD2C47104608D6004508D7
:1009C000D5000030D8007330D7009B2B2208C6001A
:1009D0002108C5004718EE2C0310EF2C0314C60C99
:1009E000C50C4718F52C0310F62C0314C60CC50CC7
:1009F0004718FC2C0310FD2C0314C60CC50C47181B
:100A0000032D0310042D0314C60CC50C47180A2D22
:100A100003100B2D0314C60CC50C4718112D031021
:100A2000122D0314C60CC50C4718182D0310192DD0
:100A30000314C60CC50C2030C50700300318013E56
:100A4000C6070630C50700300318013EC607450833
:100A5000C9004908D5005508803AA000803020021E
:100A60000318392D2D30D8003822FF30D506D50A8D
:100A70004B2DD6015508803AA000E4302002031C1B
:100A8000452D6430D502D60A3A2D30305607D700AE
:100A90005708D8003822D6015508803AA0008A307D
:100AA0002002031C572D0A30D502D60A4C2D3030B7
:100AB0005607D7005708D800382230305507D700DE
:100AC0005708D80038225608BA005508BB00233012
:100AD000D80038223408C6003308C5000130C700EA
:100AE000463084000008C8004808C9004708CA000A
:100AF00016234508C9004708CA001623C501450842
:100B0000C820C50AD800382204304502031D7F2DB5
:100B1000C0308B040034831605168312051E942DF5
:100B20006930C2007E22FB22C3010530C2000323CC
:100B30000330D80038226430D60023226B30D8002E
:100B400038220D30D8003822C2014208D120C20A12
:100B5000D800382228304202031DA52DC2014208C8
:100B60005520C20AD800382209304202031DAF2D99
:100B70002930D80038220D30D8003822C301053082
:100B8000C20003230330D80038226430D600232269
:100B90006B30D80038220D30D8003822CA230B120F
:100BA000C3010530C20003230B160330D8003822DE
:100BB000C101C00102304102031CE62D0230410296
:100BC000031DF12D583040020318F12D0430C200EE
:100BD000FA30D6002322C20BE82DC00A0319C10A3D
:100BE000DA2DC22DE72E0B138B138B1BF42DC001B6
:100BF0004008A320C00AD800382215304002031D47
:100C0000F82DC0014008BD20C00AD80038220630A7
:100C10004002031D022E0D30D80038220A30D800C1
:100C20003822C2017E22A108031DF72D0230C00028
:100C3000FA30D6002322C00B182EFB22242FC2012B
:100C400010304102031C282E1030C102C20A202E8F
:100C50000A3042020318332E30304207C3004308E3
:100C6000D80038223B2E41304207C3000A30C3026D
:100C70004308D80038220A3041020318462E30308B
:100C80004107C3004308D80038224E2E41304107A7
:100C9000C3000A30C3024308D80038220034C00120
:100CA00040084A20C00AD800382206304002031DFE
:100CB000502E2F08C1001F260D30D80038220A30D0
:100CC000D8003822C3012F08C40063220034F12168
:100CD0002108C3004308D80038223A3043020318E1
:100CE000762E30304302A1008A2E8A2E61304302D4
:100CF000031C812E7B3043020318812E4308DF3909
:100D0000822E4308A00041302002A0000A302007B4
:100D1000A1008A2E003467262108C2006726210818
:100D2000C100DD304102031D992E4208A100A22E10
:100D3000A22E4208A000A00EF030A0052008410716
:100D4000A100A22E00348B262108C0004008C80054
:100D5000CF212108C0004008C1001F262E2F8B265E
:100D60002108C0008B262108C1004008C3004108AB
:100D7000C4006322302F84011F30830507309F0099
:100D80008316051083120510B601B701B801B90129
:100D9000BA01BB01FF30BC00BD01BE01B101B2010F
:100DA000AE01B401B30101306600BA290230C800B7
:100DB000CF212108AD00C801CF212108AF002F08A5
:100DC000B000D82919302D02031DE72E8B2DC0014C
:100DD0004008FE20C00AD800382205304002031D1A
:100DE000E82EF1212108BF003F08D80038220D303D
:100DF000D80038220A30D800382241303F02031C84
:100E0000082F5B303F020318082F3F082038092FB6
:100E10003F08A0006D3020020319232F613020020B
:100E20000319252F2D3020020319272F2B302002E4
:100E300003192A2F7230200203192D2F7730200238
:100E400003192F2F312FF32D3A2FCA233A2FAF0337
:100E50004F263A2FAF0A4F263A2FA32E3A2FAF2E06
:100E60003A2F3F30D80038220D30D80038220A30CF
:080E7000D8003822E72E6300D0
:02400E00103F61
:08400000080002000D000F0092
:0442060000003C0078
:0242F200AF001B
:024204000900AF
:02420000CC00F0
:10420A0052006500760020003100650020000000A1
:1042D60034003600340037002E00300034004E0023
:1042E6002F00300039003000340032002E00340038
:0842F600310057005F000000D9
:00000001FF
